:100000008601850196018F288C00030E8D008312D6
:100010000B1D0F28A008031DA0030B11502803106F
:10002000930D920D910D900D051A13179618252812
:100030004B210F08D83A031D4F280E08033A031D21
:100040004F2896149401013095005520950B4F28A8
:1000500002301406031D2F28D430991931281408B2
:10006000732092064B21103084002E212F211F3047
:100070000F0503193D2896104F280310140D173E45
:10008000840010088000840A110880001A3095004E
:10009000940A141D4F2816159401F030A6008B10F9
:1000A0000D0E83008C0E0C0E090026080F39031D5F
:1000B0006B282608F039803A031972281A30A607EF
:1000C000FF30A61B6828260E0F39173E8400000853
:1000D000A7008514722827188510271C851403147F
:1000E000A70CA603080082073F3466345A346D34E7
:1000F00082072D342034383430342E3431342034D7
:100100005334443452342D3443344934503420343D
:100110002D34813486348C34A834A8348234831648
:100120004730810011308500F13086008312051CB4
:100130001616FC212430161AE2218B131622FA21FE
:100140009001910192019301A1019F017F30A000D4
:10015000B0308B006400200803199D280339031D6B
:10016000B528A00320229F0A9F13161DAA28161146
:100170007030A0041708180621060319C228961625
:10018000A106AA28961EC728961216229F011908B2
:10019000F0390319D428203A031900291908F8392D
:1001A000403A03191029AA288F30E2212030191D66
:1001B000DC282D301A1A2A30E3211A0D0639063AA6
:1001C0000319ED28063A283E8B1384001D08800091
:1001D000840A1E0880008B17AA288030E221280894
:1001E000E0212908E0212A08E0212B08E0212C0841
:1001F000E0212D08E0211D08E0211E08E021AA28A9
:100200001A0D3E39A300A3071F08A302A3131B085E
:10021000D0211C08D0211D08D0211E08D021AA28D9
:100220008930E2211D0E0F391C181038A2001E0C57
:100230000F399E1A003CA2071830A21BA207220207
:10024000031C22085A223A30E3211E0DA2001D0D84
:10025000A300220D230D3F395A22AA2816148030FC
:1002600095008E1C3A291F300F05031D3A291610E0
:100270001508800603108F0D8E0D161C45290E1DC6
:100280004529B9308F0601308E060310950C031CEA
:100290003129840A08008F018E01131F532903306E
:1002A0008E061B308F06931F592903308E068F3020
:1002B0008F06121C5F2902308E06A7308F06F7309A
:1002C00092188F06121D682901308E06EE308F06B7
:1002D000921D6E2903308E06DC308F06121E7429A3
:1002E00002308E0601308F06921E7A2901308E066A
:1002F000BB308F06121F802903308E0676308F06A2
:10030000921F862903308E0655308F06111C8C29CA
:1003100003308E0613308F06911C922903308E060F
:100320009F308F06111D982902308E0687308F0668
:10033000B73091198F06111EA12901308E066E303B
:100340008F06911EA72902308E06DC308F06013001
:10035000111B8F060230911B8F06043010188F0678
:10036000083090188F06103010198F062030901921
:100370008F064030101A8F068030901A8F06013099
:10038000101B8E060230901B8E060800043086007B
:100390008614060D8610861486100318C8290800D6
:1003A000A4002308231BDD29161ADC29273CC030B2
:1003B000031C68302307DD29903EE221A30A2408AC
:1003C0000023E3299615A200C6218316013086007A
:1003D00083122208F321220EF32196118316F130A5
:1003E000860083120800F039961D083886008614AE
:1003F000861008001130FD291630A3002303782051
:10040000A2009615A21F96117F39E321A30BFE29A6
:100410000800C6218615861406088610F039A20049
:100420008614060E86100F39220408000130E221DE
:100430004030A300E2212030E321A30B1B2A080057
:100440000430E2214030A400E2210922A3003F3021
:10045000A5005122C030161A9030A400E2210922D2
:10046000A5007F30E2212508E3212730161A3F300E
:10047000A5005122161A482A9030A400E221092230
:10048000A500E730E2212508E3211730A50051221D
:10049000A730161ACF30E2212308E3210630E221EB
:1004A0000800A40A2408E2210922E321A50B512A0D
:1004B00064000800A201F63EA20A03185B2AFA3E75
:1004C000A20E2207A300230E662223080F39063E40
:0804D0008318073E2A3EE329D0
:10060000A200A21B082BE03903192034220808009D
:100610008B1303308A000E238A01090022087F39D8
:1006200082076134613465346534693469346F3408
:100630006F3475347534EE3443345334E2346934F2
:1006400069346134E13465346534693469346F3454
:10065000EF347534F534EE34633473347134693403
:1006600069346134E03463342534473465346E349E
:100670009434F7344334ED3424347F345E347E34A0
:100680007634DF343134323433342B3449346E34FD
:10069000F534E4343F34FD34DF3420342034203466
:1006A00024344134413445344534493449344F3499
:1006B0004F34553455345234433453345A3444341B
:1006C0004C344134E13445344534493449344F34B1
:1006D000EF345534F5347234633473347A3464341B
:1006E0006C344134413445344534793459344F34D1
:1006F000303470346E345234433453345A34FA3410
:1007000064346134613465346534773479346F34FA
:10071000F23470346E347234633473347A34FA34AD
:02072000203483
:00000001FF
